:100000000C945A000C9477000C9477000C947700B1
:100010000C9477000C9477000C9477000C94770084
:100020000C9477000C9477000C9477000C94770074
:100030000C9477000C9477000C9477000C94770064
:100040000C9406010C9477000C9477000C947700C4
:100050000C9477000C9477000C9477000C94770044
:100060000C9477000C947700000024272A000025C8
:10007000282B000023262904040404040404040299
:100080000202020202030303030303010204081035
:100090002040800102040810200102040810200002
:1000A0000000070002010000030406000000000039
:1000B0000000000011241FBECFEFD8E0DEBFCDBF8F
:1000C00011E0A0E0B1E0E4E3F5E002C005900D929C
:1000D000A030B107D9F711E0A0E0B1E001C01D9256
:1000E000A830B107E1F70E94A3000C9498020C9489
:1000F0000000DF93CF9300D0CDB7DEB78A8384E0D2
:1001000061E00E94E301198216C08A81282F30E045
:100110008981882F90E0A90102C0559547958A955D
:10012000E2F7CA01982F917084E0692F0E940102C2
:1001300089818F5F89838981883038F30F900F9090
:10014000CF91DF910895DF93CF9300D0CDB7DEB785
:1001500082E060E00E94E30183E061E00E94E3014D
:100160008CE061E00E94E3018DE061E00E94E30128
:100170000E94A90182E00E944C021A8281309105FE
:1001800011F481E08A838A818823B1F08CE061E0F8
:100190000E94010288EC0E94790082E00E944C02D9
:1001A0001982009711F481E089838981882321F0E5
:1001B0008DE061E00E94010264EF71E080E090E078
:1001C0000E9471018CE060E00E9401028CE060E01E
:1001D0000E940102CFCFDF93CF93CDB7DEB783E08C
:1001E00061E00E9401026AE070E080E090E00E941D
:1001F000710183E060E00E9401026AE070E080E04B
:1002000090E00E947101CF91DF9108951F920F92AB
:100210000FB60F9211242F938F939F93AF93BF9399
:100220008091000190910101A0910201B091030120
:100230008050904CAF4FBF4F8093000190930101CD
:10024000A0930201B093030127C080910001909117
:100250000101A0910201B091030180589E43A0408A
:10026000B0408093000190930101A0930201B093EC
:1002700003018091040190910501A0910601B091C4
:1002800007010196A11DB11D809304019093050102
:10029000A0930601B09307018091000190910101A4
:1002A000A0910201B091030181589E43A040B0404B
:1002B00060F6BF91AF919F918F912F910F900FBEDC
:1002C0000F901F9018958FB7F894209104013091EA
:1002D000050140910601509107018FBFB901CA0184
:1002E0000895EF92FF920F931F937B018C018FB7BC
:1002F000F8944091040150910501609106017091BC
:1003000007018FBF2FB7F8948091040190910501E8
:10031000A0910601B09107012FBF841B950BA60B7E
:10032000B70B8E159F05A007B10760F31F910F91C2
:10033000FF90EF900895019759F0FC01EE0FFF1F19
:10034000EE0FFF1F32978FB7F8943197F1F78FBFF9
:100350000895789484B5826084BD84B5816084BD3D
:1003600085B5826085BD85B5816085BDEEE6F0E02E
:10037000808181608083E1E8F0E080818260808319
:10038000808181608083E0E8F0E08081816080830B
:10039000E1EBF0E0808184608083E0EBF0E080813D
:1003A00081608083EAE7F0E08081846080838081DF
:1003B0008260808380818160808380818068808387
:1003C0001092C1000895282F30E0C90185579F4F32
:1003D000FC01949129583F4FF9018491882381F0C1
:1003E000E82FF0E0E859FF4FE491F0E0662329F4AC
:1003F000808190958923808308958081892B8083D3
:100400000895482F50E0CA0181569F4FFC01249166
:10041000CA0185579F4FFC01949149585F4FFA01DB
:1004200034913323C1F1222331F1233021F480911F
:1004300080008F7705C0243031F4809180008F7D5B
:100440008093800018C0213019F484B58F7704C0E0
:10045000223021F484B58F7D84BD0DC0263021F477
:100460008091B0008F7705C0273029F48091B000CB
:100470008F7D8093B000E32FF0E0E359FF4FE491CC
:10048000F0E0662329F48081909589238083089584
:100490008081892B80830895482F50E0CA018156BE
:1004A0009F4FFC012491CA0185579F4FFC019491F5
:1004B00049585F4FFA013491332319F420E030E0BA
:1004C00035C0222331F1233021F4809180008F77D1
:1004D00005C0243031F4809180008F7D80938000AE
:1004E00018C0213019F484B58F7704C0223021F46C
:1004F00084B58F7D84BD0DC0263021F48091B0007D
:100500008F7705C0273029F48091B0008F7D8093CC
:10051000B000E32FF0E0EE58FF4FE491F0E080816F
:1005200020E030E0892311F021E030E0C901089596
:04053000F894FFCF6D
:00000001FF
